:100000000C9434000C9451000C9451000C94510049
:100010000C9451000C9451000C9451000C94340138
:100020000C9451000C9451000C9451000C94030159
:100030000C9451000C9451000C94D2000C9451007B
:100040000C9451000C9451000C9451000C945100EC
:100050000C9451000C9451000C9451000C945100DC
:100060000C9451000C94510011241FBECFEFD8E026
:10007000DEBFCDBF11E0A0E0B1E0E8E6F6E002C0EF
:1000800005900D92A431B107D9F711E0A4E1B1E0D8
:1000900001C01D92A931B107E1F70E9485010C94BE
:1000A00032030C940000CF92DF92EF92FF920F93F5
:1000B0001F93CF93DF93EC01C880D980EA80FB8047
:1000C00001E010E020E030E040EA50E4C701B60172
:1000D0000E94190287FD02C000E010E01D830C831E
:1000E00001E010E020E030E040E051E4C701B6015B
:1000F0000E94190287FD02C000E010E01F830E83FA
:100100008A899B898230910561F08330910599F04D
:100110000197C9F416BC80916E00826080936E00D6
:1001200016C0109285001092840080916F0082604A
:1001300080936F000CC01092B200809170008260BA
:100140008093700004C081E090E00E9432037894B4
:100150009FB7F894809116019FBF8823C9F310922E
:100160001601EC85FD858C819D81892B19F080819C
:10017000826002C080818D7F8083EE85FF858E81C5
:100180009F81892B19F08081886002C08081877FE0
:100190008083DF91CF911F910F91FF90EF90DF90BF
:1001A000CF9008951F920F920FB60F9211242F93A4
:1001B0003F938F939F938091140190911501019625
:1001C000909315018093140180911601813091F074
:1001D000209114013091150180911701909118011F
:1001E0002817390738F081E0809316011092150125
:1001F000109214019F918F913F912F910F900FBEFC
:100200000F901F9018951F920F920FB60F92112406
:100210002F933F938F939F93809114019091150199
:1002200001969093150180931401809116018130FD
:1002300091F0209114013091150180911701909156
:1002400018012817390738F081E0809316011092C1
:100250001501109214019F918F913F912F910F9052
:100260000FBE0F901F9018951F920F920FB60F920E
:1002700011242F933F938F939F938091140190911A
:100280001501019690931501809314018091160138
:10029000813091F020911401309115018091170166
:1002A000909118012817390738F081E080931601E2
:1002B00010921501109214019F918F913F912F91EF
:1002C0000F900FBE0F901F901895FC01239A85E2A6
:1002D00090E09787868725B5236025BD21E030E033
:1002E000318B208B42E050E050931801409317016E
:1002F00044B5426044BD49EF47BD338B228B219A00
:100300009587848780E090E00895CF92DF92EF9206
:10031000FF9280E091E00E946501C12CD12C760112
:1003200060E070E0CB016093000170930101809365
:1003300002019093030180E091E00E9453008FEF4F
:10034000C81AD80AE80AF80AC701B6010E941D02B5
:100350002FE632E143E05BE30E94CF0220E030E091
:10036000A9010E94B501DFCF5058BB27AA270ED0A4
:10037000DCC0CDD030F0D2D020F031F49F3F11F46A
:100380001EF4C2C00EF4E095E7FBB8C0E92FDED042
:1003900080F3BA17620773078407950718F071F4A2
:1003A0009EF5F6C00EF4E0950B2EBA2FA02D0B0192
:1003B000B90190010C01CA01A0011124FF27591BAA
:1003C00099F0593F50F4503E68F11A16F040A22FB0
:1003D000232F342F4427585FF3CF46953795279521
:1003E000A795F0405395C9F77EF41F16BA0B620B20
:1003F000730B840BBAF09150A1F0FF0FBB1F661F67
:10040000771F881FC2F70EC0BA0F621F731F841FA9
:1004100048F4879577956795B795F7959E3F08F0CF
:10042000B3CF9395880F08F09927EE0F979587958E
:10043000089540D008F481E00895E89409C097FB3E
:100440003EF490958095709561957F4F8F4F9F4FAB
:100450009923A9F0F92F96E9BB279395F6958795EF
:1004600077956795B795F111F8CFFAF4BB0F11F4B2
:1004700060FF1BC06F5F7F4F8F4F9F4F16C0882359
:1004800011F096E911C0772321F09EE8872F762F8F
:1004900005C0662371F096E8862F70E060E02AF0D0
:1004A0009A95660F771F881FDAF7880F96958795BC
:1004B00097F90895990F0008550FAA0BE0E8FEEF91
:1004C00016161706E807F907C0F012161306E40718
:1004D000F50798F0621B730B840B950B39F40A2611
:1004E00061F0232B242B252B21F408950A2609F4EF
:1004F000A140A6958FEF811D811D089597F99F67F3
:1005000080E870E060E008959FEF80EC089500249B
:100510000A941616170618060906089500240A9468
:1005200012161306140605060895092E0394000CEE
:1005300011F4882352F0BB0F40F4BF2B11F460FF7D
:1005400004C06F5F7F4F8F4F9F4F089557FD9058A6
:10055000440F551F59F05F3F71F04795880F97FB87
:10056000991F61F09F3F79F0879508951216130641
:100570001406551FF2CF4695F1DF08C01616170670
:100580001806991FF1CF86957105610508940895A5
:10059000E894BB2766277727CB0197F908950BD0FE
:1005A000C4CFB5DF28F0BADF18F0952309F0A6CF45
:1005B000ABCF1124EECFCADFA0F3959FD1F3950FF7
:1005C00050E0551F629FF001729FBB27F00DB11DD7
:1005D000639FAA27F00DB11DAA1F649F6627B00D67
:1005E000A11D661F829F2227B00DA11D621F739F50
:1005F000B00DA11D621F839FA00D611D221F749F5E
:100600003327A00D611D231F849F600D211D822FA4
:10061000762F6A2F11249F5750408AF0E1F08823EB
:100620004AF0EE0FFF1FBB1F661F771F881F9150F8
:100630005040A9F79E3F510570F060CFAACF5F3FB1
:10064000ECF3983EDCF3869577956795B795F7952B
:10065000E7959F5FC1F7FE2B880F911D96958795B3
:0806600097F90895F894FFCF0B
:1006680000000000010001006F12033B00000000C1
:04067800000000007E
:00000001FF
